:040000000200333295
:03000B0002005D93
:0100130032BA
:01001B0032B2
:03002300020118BF
:01002B0032A2
:0D00330075810F120280E582600302005803
:0A0040007533007534007535007546
:09004A0036007537FA75380075AF
:050053003901753A00BF
:0500580012023280FEDF
:0E005D00C0E0C0F0C082C083C0D075D00805DE
:05006B003AE53A7003C4
:03007000753300E5
:06007300153BE53B7002A5
:02007900D2961D
:0C007B006390800538E538600302010D39
:08008700853738E534700302EF
:02008F00010D61
:09009100E534B40104740180019E
:01009A00E481
:03009B00FA6015F3
:03009E0030941289
:0B00A100E53925E0F539C374089539F6
:0200AC005018EA
:0500AE0075390180130B
:0300B30030951075
:0500B600E539B401056D
:0500BB00753908800604
:0600C000E539C313F53918
:0300C600EA6013DA
:0300C90020941070
:0500CC00E536B4030558
:0500D1007534028006F9
:0600D600753400753500D1
:0500DC00E534B402133D
:0300E10020951057
:0500E400E536B4030540
:0500E9007534018006E2
:0600EE00753400753500B9
:0400F400E535600985
:0600F8001535E53570032B
:0300FE0075340056
:0C0101005390F0E5394290753B10C29617
:0B010D00D0D0D083D082D0F0D0E03200
:0E011800C0E0C0F0C082C083C002C003C0D0EF
:0901260075D000209803020223A9
:09012F00753A00C298E533600E38
:07013800E533B40102800C65
:07013F00E533B4020F800A52
:050146008599308008DE
:05014B008599318003DD
:030150008599325C
:0C0153000533C3740295334003020223FD
:0A015F00753300E53060030202234F
:0A016900C3E53194015003020203C4
:0A017300C374079531500302020324
:0C017D00E53124FFFA25E02A9001897387
:0A01890002019E0201B20201C6024B
:0901930001D10201DC0201EB02C2
:02019C0001F66A
:07019E00853235E5356005EF
:0501A500753401800328
:0301AA00753400A9
:0501AD007536008051D1
:0701B200853235E5356005DB
:0501B900753402800313
:0301BE0075340095
:0501C100753600803DD1
:0B01C60075340175350075360180327C
:0B01D10075340275350075360280277A
:0401DC00E534700393
:0301E00075340172
:0801E300753603753500801824
:0B01EB00753400753600753500800D7E
:0701F600853237C3E538959F
:0301FD0037500375
:0302000085373807
:030203003099FD32
:0D020600C299A294B3E433FA25E025E02567
:0D02130034FAA295B3E433FBC40354F8FBA6
:030220002AF59923
:0E022300D0D0D003D002D083D082D0F0D0E073
:01023100329A
:0E023200438780758BFA758DFA53890F4389C7
:0E02400020D28E759840439810439802D2AC9D
:0E024E005389F0758CFF758A40D28CD2A9D2EC
:0E025C00AF5390F0D296A294B3E433FA25E0AB
:0D026A0025E02534FAA295B3E433FBC4036C
:0602770054F8FB2AF59982
:02027D0080FE01
:01027F00225C
:0302800075820084
:010283002258
:00000001FF
